:100000000C942A000C9447000C9447000C94470071
:100010000C9447000C9447000C9447000C94470044
:100020000C9447000C9447000C9447000C94470034
:100030000C9447000C9447000C9447000C94470024
:100040000C94D8030C9447000C9447000C94470080
:100050000C94470011241FBECFE5D8E0DEBFCDBF12
:1000600010E0A0E6B0E0E8EEFDE002C005900D92E1
:10007000A236B107D9F710E0A2E6B0E001C01D92A8
:10008000A639B107E1F70E940E040C94F2060C9415
:100090000000CF93DF93EC018430910509F4A0C1F7
:1000A0008530910580F48130910509F466C0813076
:1000B0009105D0F08230910509F494C08330910508
:1000C00009F0A1C2EFC08630910509F4CDC1863098
:1000D000910508F4A7C18730910509F426C288303C
:1000E000910509F090C289C28FEF93E0909361006F
:1000F000809360006430710541F4E1E9F0E08081B3
:100100008260808320E030E0C7C26530710541F431
:10011000E2E9F0E080818260808320E030E0BCC2D0
:100120006630710541F4E3E9F0E08081826080830C
:1001300020E030E0B1C26730710541F4E4E9F0E05D
:1001400080818260808320E030E0A6C260507140F0
:1001500009F059C2A1E9B0E08C918260FD01819360
:10016000808182608083FD013296808182608083FD
:1001700013968C9182608C9346C28FEF93E090939C
:100180006100809360006430710529F41092910041
:1001900020E030E081C26530710529F410929200B0
:1001A00020E030E079C26630710529F410929300A6
:1001B00020E030E071C26730710529F4109294009C
:1001C00020E030E069C26050714009F01CC2A1E932
:1001D000B0E0FD011192108212961C9212971396B4
:1001E0001C9211C28FEF93E09093610080936000A6
:1001F0006430710541F4E1E9F0E080818160808341
:1002000020E030E049C26530710541F4E2E9F0E0F8
:1002100080818160808320E030E03EC266307105DD
:1002200041F4E3E9F0E080818160808320E030E008
:1002300033C26730710541F4E4E9F0E08081816008
:10024000808320E030E028C2E1E060307E0799F44E
:10025000A1E9B0E08C918160FD0181938081816092
:100260008083FD01329680818160808313968C911A
:1002700081608C93C8C1F2E060307F0708F4C3C18D
:10028000CB01805092409093610080936000A1E97F
:10029000B0E0FD011192108212961C9212971396F3
:1002A0001C92B1C160FF1AC041E850E029E830E07B
:1002B000D9018D919D91FA01819391938D919C919A
:1002C00091838083F90184819581FA0195838483E8
:1002D000F90186819781FA019783868363FF30C095
:1002E00080919100882341F080917000909171007D
:1002F000909382008093810080919200882341F046
:100300008091740090917500909384008093830095
:1003100080919300882341F080917800909179003A
:10032000909386008093850080919400882341F00B
:1003300080917C0090917D0090938800809387004D
:1003400061FF26C080919100882329F0E3E5F0E069
:1003500080818062808380919200882329F0EFE47D
:10036000F0E080818068808380919300882329F069
:10037000EFE4F0E0808180628083809194008823A4
:1003800009F441C1E5E4F0E08081806280833BC1F3
:1003900062FF39C180919100882329F0E3E5F0E004
:1003A00080818F7D808380919200882329F0EFE403
:1003B000F0E080818F77808380919300882329F0FB
:1003C000EFE4F0E080818F7D80838091940088232A
:1003D00009F419C1E5E4F0E080818F7D808313C1C9
:1003E00080919100882321F07093820060938100B6
:1003F00080919200882321F07093840060938300A1
:1004000080919300882321F070938600609385008B
:1004100080919400882309F4F6C07093880060935B
:100420008700F1C080919100882321F070938A00A9
:100430006093890080919200882321F070938C0052
:1004400060938B0080919300882321F070938E003D
:1004500060938D0080919400882309F4D4C0709338
:10046000900060938F00CFC064307105A9F4EEE670
:10047000F0E0208131818081918187709070906857
:10048000220F331F22953295307F3227207F32276B
:100490002070282B392B00C165307105A9F4E2E7E3
:1004A000F0E0208131818081918187709070906827
:1004B000220F331F22953295307F3227207F32273B
:1004C0002070282B392BE8C066307105A9F4E6E7C7
:1004D000F0E02081318180819181877090709068F7
:1004E000220F331F22953295307F3227207F32270B
:1004F0002070282B392BD0C06730710509F083C0DC
:10050000EAE7F0E0208131818081918187709070ED
:100510009068220F331F22953295307F3227207F3B
:1005200032272070282B392BB7C064307105B9F4FD
:10053000E0E7F0E0208131813297808191818770FE
:10054000907088609068220F331F22953295307F1B
:100550003227207F32272070282B392B9DC0653011
:100560007105B9F4E4E7F0E02081318132978081B0
:1005700091818770907088609068220F331F229558
:100580003295307F3227207F32272070282B392B5D
:1005900083C066307105B9F4E8E7F0E0208131816D
:1005A0003297808191818770907088609068220F67
:1005B000331F22953295307F3227207F32272070DB
:1005C000282B392B69C067307105E9F4ECE7F0E0BE
:1005D000208131813297808191818770907088600D
:1005E0009068220F331F22953295307F3227207F6B
:1005F00032272070282B392B4FC0CB01049704974A
:1006000008F44FC051C0CE010397039708F042C0D1
:10061000A1E9B0E08C918270FD01819380818270AC
:100620008083FD01329680818270808313968C9145
:1006300082708C938091600090916100F3E08F3F15
:100640009F0741F101969093610080936000843090
:10065000910531F481E08093910020E030E01CC0EE
:100660008530910531F481E08093920020E030E004
:1006700013C08630910531F481E08093930020E02F
:1006800030E00AC0079731F481E08093940020E0C5
:1006900030E002C020E030E0822F932FDF91CF9135
:1006A000089523E130E8F8CF20E030E0F5CF282F9F
:1006B00080916600882321F522230CF445C081E057
:1006C00080936600822F859585958595992787FD6E
:1006D00090959093650080936400332727FD3095B3
:1006E000277030708091620090916300887F282B82
:1006F000392B309363002093620020E030E026C065
:1007000010926600222304F5622F772767FD70950B
:100710006F777070660F771F660F771F660F771FF2
:10072000809162009091630087709070682B792BA4
:100730007093630060936200809164009091650003
:100740000E9449009C0102C020E030E0822F932FDC
:1007500008958CEC86B920E030E04EE650E0C90107
:10076000880F991FFA01E80FF91F118210822F5F7D
:100770003F4F2830310599F708951CBE13BC1BBCB0
:100780001ABC19BC18BC8BE483BF81E08FBD8BE021
:100790008EBD8CE485BD0895FC01E770F070EE0F0E
:1007A000FF1FE259FF4F20813181822F932F08953F
:1007B0001F920F920FB60F9211242F933F938F9396
:1007C0009F93AF93BF93EF93FF93A7E2B0E08C9119
:1007D00090E08770907024B135B1FC01EE0FFF1FDF
:1007E000E259FF4F31832083019687708C93E6E2B4
:1007F000F0E08081806480838C91882311F41092D2
:100800007E00FF91EF91BF91AF919F918F913F91AA
:100810002F910F900FBE0F901F9018952F923F921F
:100820004F925F926F927F928F929F92AF92BF9200
:10083000CF92DF92EF92FF920F931F93CF93DF93AC
:100840001ABA88EF87BB8FEF84BB80EF81BB18BAE1
:100850001CBE1BBC1ABC19BC18BC13BCE3E5F0E001
:1008600080818F7D8083EFE4F0E080818F778083CB
:1008700080818F7D8083E5E4F0E080818F7D8083BF
:10088000E5E3F0E080818260808380818E7F8083D9
:1008900080818860808380818B7F8083808180627B
:1008A000808380818F7E8083808180688083808147
:1008B0008F7B808387E690E00E94B3060E94A903A5
:1008C0000E94BD03789410927E00662477248824C9
:1008D0009924AA24BB24CC24DD2405E310E00F2EA8
:1008E000F0E72F2EF0E03F2EF02D0F2EF8E3EF2E45
:1008F000FF24F02D44245524F4C0EBE2F0E0808185
:1009000088235CF40E94BC060E945703EC01009708
:1009100021F00E94C306D0936D00EBE2F0E08081ED
:1009200085FF08C080916D00882321F00E94C306D6
:1009300010926D00E3E5F0E0808185FD07C0F801CD
:100940008081F3E08F27F801808328C0F101808146
:100950009181208131818150934064F02F3F310596
:1009600009F044F4F80180818260808380818E7F69
:10097000808314C0ECE5F0E08081813440F0F80120
:1009800080818E7F808380818D7F808307C0F80186
:1009900080818160808380818D7F8083EFE4F0E0BF
:1009A000808188233CF0F8018081FCE08F27F801EA
:1009B00080832BC0E4E7F0E0808191812081318148
:1009C0008150934064F02F3F310509F044F4F80161
:1009D00080818860808380818B7F808316C0EAE479
:1009E000F0E0808191818134910540F0F8018081AF
:1009F0008B7F80838081877F808307C0F80180811F
:100A0000846080838081877F8083EFE4F0E0808151
:100A100085FD07C0F8018081F0E38F27F80180830E
:100A20002BC0E8E7F0E08081918120813181815005
:100A3000934064F02F3F310509F044F4F8018081C0
:100A40008062808380818F7E808316C0E8E4F0E03E
:100A5000808191818134910540F0F80180818F7E01
:100A6000808380818F7D808307C0F80180818061D1
:100A7000808380818F7D8083E5E4F0E0808185FD47
:100A800007C0F8018081F0EC8F27F801808329C02E
:100A9000ECE7F0E0808191812081318181509340A9
:100AA00064F02F3F310509F044F4F801808180683B
:100AB000808380818F7B808314C0E3E4F0E08081B9
:100AC000813440F0F80180818F7B808380818F7733
:100AD000808307C0F80180818064808380818F7764
:100AE000808380917E00882309F007CFF101808107
:100AF0009181E1E8F0E020813181281B390BC901A7
:100B000085529F4F875B914010F0620113C0C60170
:100B1000820F931F4FEF8432940714F484E29FEF07
:100B20006C018DEDC816D1042CF00F2EFCEDCF2EEC
:100B3000DD24F02DC601DD200CF4039695958795F4
:100B400095958795280F391FA90133231CF45095DB
:100B500041955F4F4F3F510519F014F08FEF04C0DE
:100B600055230CF4A201842FECE5F0E080831216EB
:100B700013062CF4F70180818061808304C0F701A3
:100B800080818F7E8083E4E7F0E080819181E3E8DB
:100B9000F0E020813181281B390BC90185529F4F1C
:100BA000875B914010F0520113C0C501820F931F63
:100BB0004FEF8432940714F484E29FEF5C018DEDD3
:100BC000A816B1042CF00F2EFCEDAF2EBB24F02D97
:100BD000C501BB200CF4039695958795959587954F
:100BE000280F391FA90133231CF4509541955F4FFD
:100BF0004F3F510521F01CF04FEF50E003C055234B
:100C00000CF4A201EAE4F0E05183408312161306CB
:100C10002CF4F70180818062808304C0F701808119
:100C20008F7D8083E8E7F0E080819181E5E8F0E066
:100C300020813181281B390BC90185529F4F875B69
:100C4000914010F0420113C0C401820F931F4FEF77
:100C50008432940714F484E29FEF4C018DED8816E2
:100C600091042CF00F2EFCED8F2E9924F02DC40151
:100C700099200CF403969595879595958795280F5F
:100C8000391FA90133231CF4509541955F4F4F3F05
:100C9000510521F01CF04FEF50E003C055230CF438
:100CA000A201E8E4F0E051834083121613062CF40D
:100CB000F70180818064808304C0F70180818F7B8D
:100CC0008083ECE7F0E080819181E7E8F0E020812B
:100CD0003181281B390BC90185529F4F875B914099
:100CE00010F0320113C0C301820F931F4FEF843203
:100CF000940714F484E29FEF3C018DED68167104B3
:100D00002CF00F2EFCED6F2E7724F02DC3017720F1
:100D10000CF403969595879595958795280F391F1F
:100D2000A90133231CF4509541955F4F4F3F510566
:100D300019F014F08FEF04C055230CF4A201842F96
:100D4000E3E4F0E08083121613062CF4F7018081AF
:100D50008068808304C0F70180818F778083F1E011
:100D6000F0937E00BECEE0E4F0E0908389B988E1A4
:100D70008AB98EE880830895EBE2F0E080818823D1
:100D8000ECF78CB10895982FEBE2F0E0808185FFBD
:100D9000FDCF9CB908951F93282F82958F70982FAF
:100DA000905D9A3308F0995F822F8F70182F105D35
:100DB0001A3308F0195F892F0E94C306812F0E9401
:100DC000C3061F910895CF93DF93EC018881882398
:100DD00031F00E94C306219688818823D1F7DF91E4
:080DE000CF910895F894FFCFB4
:020DE800FF0307
:00000001FF
